:10000000C328A8008417800484138E010C1C8E0062
:1000100023200319BE2823200319BE282320BE282D
:10002000A80059200C080D040319BE28B820841319
:100030002808800664001C281D288C0A03198D0FCF
:100040001A288006BE2828088E0601308C008D01F3
:10005000000828050E06031D08008C0A03198D0FE1
:10006000282808008F002A08840028095A208413B1
:100070008F080319BE28F03091000E0880389000D8
:10008000F03091030319910003198F030319BE285F
:1000900049285D2003010C1828088E1F28088E08A7
:1000A00003190301900F562880063D2857280000A9
:1000B0004028FF3A84178005BE280D080C04031958
:1000C0008C0A80300C1A8D060C198D068C188D0642
:1000D0000D0D8C0D8D0DBE288F018E00FF308E070B
:1000E000031C8F07031CBE2803308D00DF307A20ED
:1000F0006E288D01E83E8C008D09FC30031C83289E
:100100008C07031880288C0764008D0F80280C183A
:1001100089288C1C8D2800008D2808008D018F01F6
:100120008E0002309D288D018F018E0001309D28A8
:100130008D018F018E0004309D2894000F080D0260
:10014000031DA4280E080C02043003180130031903
:1001500002301405031DFF30BE280038031DFF3098
:100160000405031DFF30BE280404031DFF30BE2814
:100170008C098D098C0A03198D0A08008313031357
:10018000831264000800831603308500083086005F
:1001900083128610831686108312061083160610AB
:1001A00006308312AA001030A80064308E000A3096
:1001B000322032308E000530322046308E000A3038
:1001C000322032308E000230322001308C00053077
:1001D0008400013001200C08AC0001308C00053097
:1001E0008400023001200C08AD002C088C009B30EC
:1001F00093209E002C088C0091309820A0001E08AF
:1002000084002008B420A000A1002D088C009B30A1
:100210009320A2002D088C0091309820A400220881
:1002200084002408B420A400A50020082104840030
:1002300024082504B420A400A50064002408250493
:1002400003192B290630AA001030A80064308E0054
:1002500005303220E52801308C0005308400013063
:1002600001200C08AC0001308C0005308400023005
:1002700001200C08AD002C088C0000308E209E0060
:100280002D088C0000308E20A0001E08840020085D
:10029000B420A000A1006400200821040319512902
:1002A000E5282D088C00B43093209E002C088C008B
:1002B00091309320A0002C088C009B309820A20045
:1002C000200884002208AD20A200A3001E0884009C
:1002D00022082304AD20A200A30064002208230406
:1002E0000319732932222D088C00783098209E0043
:1002F0002C088C0091309320A0002C088C009B309F
:100300009820A200200884002208AD20A200A300AB
:100310001E08840022082304AD20A200A30064006C
:10032000220823040319952943222C088C007830D5
:1003300098209E002D088C0091309320A0002D085D
:100340008C009B309820A200200884002208AD2059
:10035000A200A3001E08840022082304AD20A200EE
:10036000A3006400220823040319B72965222C087E
:100370008C00B43093209E002D088C009130932087
:10038000A0002D088C009B309820A200200884003B
:100390002208AD20A200A3001E0884002208230426
:1003A000AD20A200A3006400220823040319D92968
:1003B00054222C088C00783098209E002D088C0048
:1003C000B4309320A0001E0884002008AD20A000B7
:1003D000A1006400200821040319EF2976222C08CB
:1003E0008C00B43093209E002D088C00B4309320F4
:1003F000A0001E0884002008AD20A000A100640019
:10040000200821040319052A87222C088C00783043
:1004100098209E002D088C0078309820A0001E089F
:1004200084002008AD20A000A10064002008210461
:1004300003191B2A98222C088C00B43093209E00AC
:100440002D088C0078309820A0001E088400200819
:10045000AD20A000A1006400200821040319312A66
:10046000A9222B29AA30AF00BA22A030AE00A030BA
:10047000B000BA226430AF00BA227830AE007830D3
:10048000B000BA220800AA30AF00BA227830AE001D
:100490007830B000BA226430AF00BA22A030AE008B
:1004A000A030B000BA220800AA30AF00BA227830DB
:1004B000AE00A030B000BA226430AF00BA22A03043
:1004C000AE007830B000BA220800AA30AF00BA22DD
:1004D000A030AE007830B000BA226430AF00BA224B
:1004E0007830AE00A030B000BA220800AA30AF00C9
:1004F000BA22A030AE008C30B000BA226430AF0017
:10050000BA227830AE008230B000BA220800AA3099
:10051000AF00BA228C30AE00A030B000BA226430F6
:10052000AF00BA228230AE007830B000BA220800A4
:10053000AA30AF00BA228230AE007830B000BA22C2
:100540006430AF00BA228C30AE00A030B000BA22C6
:100550000800AA30AF00BA227830AE008230B00076
:10056000BA226430AF00BA22A030AE008C30B000A6
:10057000BA2208000130B10064000B3031020318C8
:10058000DA2A2F088C008D0106308400803010207C
:100590002E088C008D010630840040301020300879
:1005A0008C008D0106308400203010200D306C202E
:0A05B000B10FBC2A08006300DB2A2B
:02400E00F53F7C
:00000001FF
